:020000040000FA
:02000000FD28D9
:08000800CE288C008101831653
:100010000313C030810508008C008101831603138F
:10002000C030810501308104831203130B110B1DB5
:1000300017288C0B162808008E00E13086050E0D5F
:100040001E398604080086132628861706138F009B
:100050000F080F0E1C2033200F081C203320E13026
:1000600086058613080002300C20861600008612D2
:1000700002300C20080011089200931164308D00AA
:100080004C2025200A308D004C20252001308D0089
:1000900093154C20252008008C010D081202031C2A
:1000A00056288C0A0D08920293154E2830300C0702
:1000B000931D203008009400051008308C006C203F
:1000C00014180514141C0510940C6C208C0B60285B
:1000D00005146C206C2008001D308D00722808303B
:1000E0008D0072288D0B722808009501F2289A0164
:1000F0009B0106309C000800C530232015082520F0
:10010000CD302320150891003B2009305B20723050
:100110005B2065305B2063305B2065305B2069309D
:100120005B2076305B2065305B2064305B202030C4
:100130005B2015085B2020305B206F305B206E3029
:100140005B2020305B204D305B2069305B206330CA
:100150005B2072305B206F305B2063305B20683047
:100160005B2069305B2070305B2020305B2050309A
:100170005B2049305B2043305B2031305B203630E0
:100180005B2046305B2038305B2034305B200D3004
:100190005B200A305B2013100B1608008B138B1B9F
:1001A000CE289600030E970083010A0898008A0162
:1001B0008313040899008B18DE28F4280B126F2093
:1001C0000618752808308C006C2006189517061C38
:1001D00095130C0B950C8C0BE4286C20061C7528D1
:1001E0001314F3280B168B101908840018088A00C2
:1001F000170E8300960E160E0900831603130130A6
:10020000860583120313861206138613E1308605D2
:1002100008300C2003301C20332002300C20083022
:100220001C20332002300C2002301C2033200230EE
:100230000C20283023200C302320013023200830CC
:100240000C208316031305100614011383120313E5
:1002500005148B100B168B17930152302520533049
:100260002520323025203330252032302520203003
:100270002520433025206F3025206D3025206D301E
:100280002520753025206E302520693025206330EB
:100290002520613025202D302520C03023207430CA
:1002A0002520693025206F3025206E302520203014
:1002B00025206F3025206E3025202030252050301D
:1002C0002520493025204330252031302520363067
:1002D0002520463025203830252034302520303068
:1002E000900002308A001008303C08225B20900BFE
:1002F00071291A3005200730132061305B206E30E1
:100300005B2069305B206D305B2061305B20743096
:100310005B2069305B206E305B2067305B202030D3
:100320005B204C305B2043305B2044305B202E3020
:100330005B202E305B202E305B200D305B200A309E
:100340005B201030900018302320C0300C20900B20
:10035000A32901302320523025205330252032306C
:1003600025203330252032302520203025205230E2
:10037000252065302520633025206530252070300C
:10038000252074302520693025206F3025206E30DF
:1003900025203A302520C0302320433025206830E6
:1003A00025206130252072302520C730232056308B
:1003B0002520613025206C302520753025206530C2
:1003C000252072305B2065305B2061305B2064301B
:1003D0005B2079305B202E305B202E305B202E306E
:1003E0005B200D305B200A305B20772013187720CC
:1003F00013187C209A0BF6299B0BF6299C0BF629E7
:1004000040305B200D305B200A305B207720F629DE
:1004100082070D340A344D346934633472346F34D6
:10042000633468346934703420345034493443348C
:1004300031343634463438343434203463346F3411
:100440006E346E346534633474346534643420340B
:1004500061346E34643420347334743461346E34F3
:1004600064342D34623479342E342E342E340D34E9
:020470000A344C
:02400E00F13F80
:00000001FF
